:100000000C942E000C94740C0C944B000C944B002C
:100010000C944B000C944B000C944B000C944B0034
:100020000C944B000C944B000C944B000C944B0024
:100030000C944B000C944B000C944B000C944B0014
:100040000C944B000C944B000C944B000C944B0004
:100050000C944B000C944B000C944B0011241FBECD
:10006000CFEFD8E0DEBFCDBF12E0A0E0B1E0E4E525
:10007000FFE102C005900D92AA38B107D9F712E04E
:10008000AAE8B2E001C01D92AD3AB107E1F70E94C3
:10009000090D0C94A80F0C940000FF920F931F936E
:1000A000CF93DF9309E912E0CAE0D0E0FF24F39494
:1000B000CE010E94830F81508E3F18F4F801F08228
:1000C00002C0F801108221960F5F1F4FC131D10588
:1000D00079F7C1E1D0E0CE010E94830F8F3F21F07C
:1000E000FE01EA59FD4F80832196C831D10599F769
:1000F000C8E1D0E0CE010E94830F8F3F21F0FE01C6
:10010000E857FD4F80832196CF31D10599F7DF91D4
:10011000CF911F910F91FF9008951F93109170023E
:1001200080917102E0917202833018F4FE2FF15039
:1001300002C0FE2FE25097E1899FC001112469E0BF
:1001400070E00E943B0F9B012C5F3F4FE10F2E0F91
:10015000311D8F2F86958695280F311D8F2F64E6D0
:100160000E942F0F281B3109C90167E070E00E942F
:100170003B0F80936F021F9108950E948D00809124
:100180006F02E7E7F2E0E80FF11D808180936702DC
:1001900080916F02E0EAF2E0E80FF11D8081809328
:1001A000900280916F02E9E9F2E0E80FF11D808191
:1001B0008093910208950E94BD008091910288234E
:1001C00001F190918F0250918E0240918D023091F9
:1001D0008C0220916702990F892F880F880F890F51
:1001E000850F281771F420919002942F990F892F71
:1001F000880F880F890F830F281719F48DEB8093D0
:1002000097020895999AA19A0895999AA1980895A4
:1002100080E40E94780D84E00E94840D8EE00E94AC
:10022000840D8EE00E94840D8EE00E94840D8FE18B
:100230000E94840D80E00E94840D84E00E94840D61
:1002400080E00E94840D08950E949F0D0E94A30DDE
:1002500080E40E94780D8CE10E94840D8EE10E9462
:10026000840D8EE10E94840D8EE10E94840D8EE14A
:100270000E94840D8EE10E94840D8EE10E94840D07
:100280008CE10E94840D87E00E94840D8FE00E9423
:10029000840D8FE00E94840D8FE00E94840D8FE01A
:1002A0000E94840D8FE00E94840D8FE00E94840DD7
:1002B00087E00E94840D8FE10E94840D8FE10E94EF
:1002C000840D80E00E94840D80E00E94840D80E017
:1002D0000E94840D80E00E94840D8FE10E94840DB5
:1002E0008FE10E94840D8EE10E94840D8CE10E94BA
:1002F000840D80E00E94840D80E00E94840D80E0E7
:100300000E94840D80E00E94840D88E10E94840D8B
:100310008CE10E94840D8FE00E94840D87E00E9492
:10032000840D80E00E94840D80E00E94840D80E0B6
:100330000E94840D80E00E94840D83E00E94840D61
:1003400087E00E94840D80E00E94840D80E00E947E
:10035000840D80E00E94840D80E00E94840D80E086
:100360000E94840D80E00E94840D8FE10E94840D24
:100370008FE10E94840D80E00E94840D80E00E9445
:10038000840D80E00E94840D80E00E94840D80E056
:100390000E94840D80E00E94840D87E00E94840DFD
:1003A0008FE00E94840D8FE10E94840D8FE10E94F6
:1003B000840D80E00E94840D80E00E94840D80E026
:1003C0000E94840D80E00E94840D80E00E94840DD4
:1003D00080E00E94840D08956115710521F4806804
:1003E0000E94780D08956130710519F4806C0E94A7
:1003F000780D0895CF93DF93EC0160E070E00E94E8
:10040000EC0181E00E94840D87E00E94840D80E071
:100410000E94840DCE0161E070E00E94EC0181E059
:100420000E94840D85E00E94840D80E00E94840D6E
:10043000DF91CF910895CF93DF93EC0160E070E0FE
:100440000E94EC0180E20E94840D80E20E94840DF3
:1004500080E00E94840DCE0161E070E00E94EC011A
:1004600080E20E94840D80E20E94840D80E00E9460
:10047000840DDF91CF910895CF93DF93EC0160E07D
:1004800070E00E94EC0184E00E94840D82E00E94F2
:10049000840D80E00E94840DCE0161E070E00E9436
:1004A000EC0181E00E94840D85E00E94840D85E0CE
:1004B0000E94840DDF91CF910895CF93DF93EC01DB
:1004C00060E070E00E94EC0184E00E94840D82E014
:1004D0000E94840D80E00E94840DCE0161E070E0F6
:1004E0000E94EC0186E00E94840D85E00E94840D4C
:1004F00080E00E94840DDF91CF910895CF93DF9328
:10050000EC0160E070E00E94EC0181E00E94840D4B
:1005100085E00E94840D80E00E94840DCE0161E0A0
:1005200070E00E94EC0180E20E94840D80E20E9453
:10053000840D80E00E94840DDF91CF910895CF93C8
:10054000DF93EC0160E070E00E94EC0181E00E942A
:10055000840D82E00E94840D83E00E94840DCE0110
:1005600061E070E00E94EC0186E00E94840D85E06D
:100570000E94840D80E00E94840DDF91CF91089548
:10058000CF93DF93EC0160E070E00E94EC0181E02A
:100590000E94840D82E00E94840D83E00E94840DFD
:1005A000CE0161E070E00E94EC0181E00E94840DC8
:1005B00085E00E94840D80E00E94840DDF91CF9140
:1005C0000895CF93DF93EC0160E070E00E94EC01AE
:1005D00081E00E94840D87E00E94840D80E00E94EB
:1005E000840DCE0161E070E00E94EC0180E20E9487
:1005F000840D80E20E94840D80E00E94840DDF91D2
:10060000CF910895CF93DF93EC0160E070E00E94FA
:10061000EC0181E00E94840D82E00E94840D80E064
:100620000E94840DCE0161E070E00E94EC0181E047
:100630000E94840D85E00E94840D80E00E94840D5C
:10064000DF91CF910895CF93DF93EC0160E070E0EC
:100650000E94EC0181E00E94840D82E00E94840DE2
:1006600080E00E94840DCE0161E070E00E94EC0108
:1006700086E00E94840D85E00E94840D80E00E9447
:10068000840DDF91CF910895CF93DF93EC0160E06B
:1006900070E00E94EC0181E00E94840D80E00E94E5
:1006A000840DCE0161E070E00E94EC0181E00E94C7
:1006B000840D80E00E94840DDF91CF9108950F9307
:1006C0001F93CF93DF93EC018B01009721F4CB01B3
:1006D0000E94FA011CC08130910521F4CB010E94D7
:1006E0001B0215C08230910521F4CB010E943C020F
:1006F00015C08330910521F4CB010E945D021CC01E
:100700008430910521F4CB010E947E021CC0C530CB
:10071000D10521F4C8010E949F021CC0C630D1053A
:1007200021F4C8010E94C0021BC0C730D10521F4CA
:10073000C8010E94E10214C0C830D10521F4C801EB
:100740000E9402030DC0C930D10521F4C8010E94E6
:10075000230306C0CC30D10519F4C8010E9444031C
:10076000DF91CF911F910F91089580E090E00E945A
:10077000830F8093A80281E090E00E94830F809312
:10078000AA0282E090E00E94830F8093AB0283E094
:1007900090E00E94830F8093A90208950E94270F82
:1007A0008093AC020E942B0F8093A7029091AC0221
:1007B0008091A802891720F08091A8028F3F51F400
:1007C0008091AC028093A8026091A80280E090E042
:1007D0000E948B0F9091A7028091AB02891720F0A5
:1007E0008091AB028F3F51F48091A7028093AB02BE
:1007F0006091AB0282E090E00E948B0F9091AC027E
:100800008091AA02981720F08091AA028F3F51F49C
:100810008091AC028093AA026091AA0281E090E0EC
:100820000E948B0F9091A7028091A902981720F047
:100830008091A9028F3F51F48091A7028093A90271
:100840006091A90283E090E00E948B0F08951F93AE
:10085000182F80918F0290E060E070E00E945F03AB
:1008600080918E0290E063E070E00E945F038CE074
:1008700090E067E070E00E945F0380918D0290E05D
:100880006AE070E00E945F0380918C0290E06DE06E
:1008900070E00E945F03112311F00E94CE031F91AC
:1008A0000895982F92959F70990F292F220F220F4C
:1008B000290F8F70820F08956AE00E942F0F829592
:1008C000807F890F08951F93DF93CF930F92CDB749
:1008D000DEB7182F69830E940A0E0E94130E82EA67
:1008E0000E942C0E812F0E942C0E6981862F0E945F
:1008F0005C040E942C0E0E941D0E0F90CF91DF9180
:100900001F9108951F93DF93CF930F92CDB7DEB75A
:10091000182F0E940A0E0E94130E82EA0E942C0ECB
:10092000812F0E942C0E0E941D0E0E94130E83EA3E
:100930000E942C0E80E00E945E0E89830E941D0E94
:1009400089810F90CF91DF911F910895EF92FF92CF
:100950000F931F9380918B0290918A02E0908D02F9
:10096000F0908C0200918F0210918E02880F682FF8
:10097000660F660F680F690F82E00E946304EE0C39
:100980006E2D660F660F6E0D6F0D83E00E9463047F
:10099000000F602F660F660F600F610F84E00E94EA
:1009A00063046091700285E00E94630460916F02AD
:1009B00086E00E9463046091710287E00E946304F4
:1009C0006091720288E00E9463041F910F91FF9072
:1009D000EF900895CF92DF92EF92FF920F931F93C3
:1009E00084E00E948204D82E83E00E948204E82ED4
:1009F00082E00E948204F82E85E00E948204182F73
:100A000086E00E948204C82E87E00E948204082F9C
:100A100088E00E9482042D2D30E02073307064E065
:100A2000359527956A95E1F7220F422F440F440F21
:100A3000420F9D2D9F70490F2E2D30E02077307092
:100A400054E0359527955A95E1F7220F522F550F0F
:100A5000550F520F9E2D9F70590F2F2D30E020778C
:100A6000307094E0359527959A95E1F7220F922FF3
:100A7000990F990F920F2F2D2F70920F382F3295BB
:100A80003F70330F232F220F220F230F8F70280F59
:100A900020937202202F2695269526952271822F6B
:100AA000880F880F820F0F70800F809371028C2D3A
:100AB000877080936F02212F30E02073307084E0C4
:100AC000359527958A95E1F7220F822F880F880F99
:100AD000820F1F70810F809370022AE0892F622F8E
:100AE0000E942F0F80938B0290938A02852F0E9481
:100AF0002F0F80938D0290938C02842F0E942F0FD2
:100B000080938F0290938E021F910F91FF90EF9030
:100B1000DF90CF9008958CE00E94D30D0E940201D7
:100B20005198599AE89AE9E6F0E0808182608083E2
:100B300078940E940A0E0E94130E82EA0E942C0EE4
:100B40008DE00E942C0E83E80E942C0E0E941D0E48
:100B500052985A9A53985B9A54985C9A55985D9A11
:100B6000259A82EC809380008AE180938100109224
:100B700087001092860084EF91E090938900809323
:100B800088000E94EA040E944D000E94B5030E9462
:100B9000BD000E94CE030895882369F088EE93E09B
:100BA000909387008093860084EF91E09093890072
:100BB000809388000895109287001092860010920A
:100BC00089001092880008954A9919C08FE798E328
:100BD000A1E081509040A040E1F700C000004A9B96
:100BE0000AC00BC08FEF99EFA0E081509040A04069
:100BF000E1F700C000004A9BF5CF81E0089580E056
:100C000008954B990EC08FE798E3A1E08150904082
:100C1000A040E1F700C0000081E04B9B03C080E0F2
:100C2000089580E008954C990EC08FE798E3A1E005
:100C300081509040A040E1F700C0000081E04C9B53
:100C400003C080E0089580E008951092940210920D
:100C50009302809192028F5F809392028091920220
:100C6000873010F01092920208954D992DC08FE7B1
:100C700098E3A1E081509040A040E1F700C000005F
:100C80004D9919C080919702843099F414C08FEF68
:100C900099EFA0E081509040A040E1F700C0000033
:100CA0008091930290919402019690939402809384
:100CB00093024D9BECCF80919302909194028333E9
:100CC000910520F00E94250680E0089581E00895B6
:100CD00080919702882329F580918E028F5F8093FF
:100CE0008E0280918E028A3038F010928E028091AE
:100CF0008F028F5F80938F0280918F02823040F04D
:100D000080918E02843020F010928E0210928F0219
:100D100010928A0210928B0280E00E9427040E94A7
:100D2000A60480919702843021F5809170028F5F34
:100D30008093700280917102823059F0909170021C
:100D4000E0917102F0E0E358FD4F8081891788F44B
:100D50000DC080917202837029F0809170028D31F4
:100D600040F004C0809170028E3118F081E08093D1
:100D70007002809197028D3B29F41092970280E0D7
:100D80000E94CC0580919702853051F5E091920246
:100D9000F0E0E958FD4F80818F5F8083E0919202FF
:100DA000F0E0E958FD4F8081883130F0E091920207
:100DB000F0E0E958FD4F1082E0919202F0E0E9582E
:100DC000FD4F808180936A0280919202E0919202AD
:100DD00090E0F0E0E958FD4F419660810E948B0F52
:100DE0000895809197028823F9F480918C028F5F97
:100DF00080938C0280918C028A3038F010928C02A1
:100E000080918D028F5F80938D0280918D0286305C
:100E100010F010928D0210928A0210928B0280E0E4
:100E20000E9427040E94A60480919702843059F5FD
:100E3000809171028F5F80937102809171028D3079
:100E400018F081E08093710280917102823059F034
:100E500090917002E0917102F0E0E358FD4F8081C3
:100E6000891788F40DC080917202837029F08091F7
:100E700070028D3140F004C0809170028E3118F004
:100E800081E080937002809197028D3B29F410924B
:100E9000970280E00E94CC0580919702853051F541
:100EA000E0919202F0E0E056FD4F80818F5F8083F9
:100EB000E0919202F0E0E056FD4F80818C3330F0FB
:100EC000E0919202F0E0E056FD4F1082E091920234
:100ED000F0E0E056FD4F808180936C028091920299
:100EE000E091920290E0F0E0E056FD4F489660817C
:100EF0000E948B0F089580919702843039F580917C
:100F000072028F5F8093720280917202843610F0B9
:100F10001092720280917202837051F4809171027A
:100F2000823031F4809170028E3108F44CC00AC0D6
:100F300080917102823009F046C0809170028D313B
:100F400008F441C081E08093700208958091970277
:100F50008D3B31F41092970280E00E94CC050895F9
:100F600080919702853059F5E0919202F0E0E756C2
:100F7000FD4F8081882339F0E0919202F0E0E7563E
:100F8000FD4F108207C0E0919202F0E0E756FD4F5E
:100F900081E08083E0919202F0E0E756FD4F80818E
:100FA00080936E0280919202E091920290E0F0E0D4
:100FB000E756FD4F0A9660810E948B0F089584B317
:100FC00092E0892784BB08950E94E405882381F07C
:100FD000809197028D3B51F080919702853031F0DE
:100FE000809197028F5F8093970202C010929702C0
:100FF0000E940106882311F00E9468060E941306D1
:10100000882311F00E94F1060E943506882311F012
:101010000E947B070895882369F0813071F0823047
:1010200079F0833081F0843089F0853091F086301A
:1010300099F0089520E031E011C021E131E00EC0C7
:1010400022E231E00BC023E331E008C024E431E0C8
:1010500005C025E531E002C026E631E0C90108956A
:10106000882369F0813071F0823079F0833081F02B
:10107000843089F0853091F0863099F0089527E723
:1010800031E011C02EE731E00EC027E831E00BC09F
:101090002EE831E008C025E931E005C02DE931E056
:1010A00002C024EA31E0C9010895FF920F931F9313
:1010B000DF93CF93CDB7DEB760970FB6F894DEBF5E
:1010C0000FBECDBF082FF62E8A3020F48BEA91E0B8
:1010D0000E94B90D802F90E08E010F5F1F4FB80165
:1010E0004AE050E00E94620FC8010E94B90D8DEAEB
:1010F00091E00E94B90D8F2D8A3020F48BEA91E0A7
:101100000E94B90D8F2D90E08E010F5F1F4FB80127
:101110004AE050E00E94620FC8010E94B90D60963B
:101120000FB6F894DEBF0FBECDBFCF91DF911F91F8
:101130000F91FF900895882329F00E94240181E0F7
:101140000E94270408950F931F93DF93CF93CDB789
:10115000DEB760970FB6F894DEBF0FBECDBF882311
:1011600079F00E949F0D0E94A30D8FEA91E00E94EA
:10117000B90D8BE060E00E94900D8FED0E94A70DED
:101180000E94CE0389E060E00E94900D8091AC0245
:1011900090E08E010F5F1F4FB8014AE050E00E94BF
:1011A000620FC8010E94B90D89E061E00E94900DB4
:1011B0008091A70290E0B8014AE050E00E94620FDF
:1011C000C8010E94B90D60960FB6F894DEBF0FBE3D
:1011D000CDBFCF91DF911F910F9108950F931F9372
:1011E000DF93CF93CDB7DEB760970FB6F894DEBF2D
:1011F0000FBECDBF882379F00E949F0D0E94A30DE2
:101200008BEC91E00E94B90D8EE060E00E94900DA1
:101210008FED0E94A70D8CE060E00E94900D809100
:10122000A80290E08E010F5F1F4FB8014AE050E026
:101230000E94620FC8010E94B90D8CE061E00E941B
:10124000900D8091AB0290E0B8014AE050E00E941E
:10125000620FC8010E94B90D60960FB6F894DEBF08
:101260000FBECDBFCF91DF911F910F9108950F93C6
:101270001F93DF93CF93CDB7DEB760970FB6F89487
:10128000DEBF0FBECDBF882379F00E949F0D0E9464
:10129000A30D8DEE91E00E94B90D8EE060E00E94FA
:1012A000900D8FED0E94A70D8CE060E00E94900DE4
:1012B0008091AA0290E08E010F5F1F4FB8014AE0B3
:1012C00050E00E94620FC8010E94B90D8CE061E0FD
:1012D0000E94900D8091A90290E0B8014AE050E090
:1012E0000E94620FC8010E94B90D60960FB6F89473
:1012F000DEBF0FBECDBFCF91DF911F910F9108953B
:101300000F931F93DF93CF93CDB7DEB760970FB6E0
:10131000F894DEBF0FBECDBF882309F44EC00E94F3
:101320009F0D0E94A30D0E948D000E94A604809133
:101330006F020E940B080E94B90D8FE092E00E949C
:10134000B90D8091700290E08E010F5F1F4FB801C0
:101350004AE050E00E94620FC8010E94B90D85E189
:1013600092E00E94B90D8091710290E0B8014AE0CC
:1013700050E00E94620FC8010E94B90D87E192E01F
:101380000E94B90D8091720290E0B8014AE050E0ED
:101390000E94620FC8010E94B90D80916F02809374
:1013A0007302809170028093740280917202809324
:1013B0007602809171028093750290916F02809104
:1013C0007302981799F490917002809174029817A3
:1013D00069F49091720280917602981739F4909195
:1013E000710280917502981709F44EC00E949F0DFA
:1013F0000E94A30D0E948D000E94A60480916F029E
:101400000E940B080E94B90D8FE092E00E94B90D76
:101410008091700290E08E010F5F1F4FB8014AE08B
:1014200050E00E94620FC8010E94B90D85E192E070
:101430000E94B90D8091710290E0B8014AE050E03D
:101440000E94620FC8010E94B90D87E192E00E94DC
:10145000B90D8091720290E0B8014AE050E00E941C
:10146000620FC8010E94B90D80916F0280937302D0
:101470008091700280937402809172028093760250
:10148000809171028093750260960FB6F894DEBF6A
:101490000FBECDBFCF91DF911F910F91089588238B
:1014A00009F473C00E949F0D0E94A30D0E940801C1
:1014B00080E090E060E070E00E94EC0180E00E943B
:1014C000840D8FE090E060E070E00E94EC0180E02D
:1014D0000E94840D81E060E00E94900D8BE192E01B
:1014E0000E94B90D809192020E9430080E94B90DAD
:1014F000E0919202F0E0E958FD4F808180936A020A
:10150000E0919202F0E0E056FD4F808180936C0202
:10151000E0919202F0E0E756FD4F808180936E02E9
:1015200080E061E00E94900DA0919202E091920211
:10153000B0E0A958BD4FF0E0E056FD4F8C916081BE
:101540000E94550888E061E00E94900DE0919202AF
:10155000F0E0E756FD4F8081882319F082E292E0A7
:1015600002C08AE292E00E94B90D809192028093BB
:10157000680280916A028093690280916C02809374
:101580006B0280916E0280936D029091680280914F
:101590009202981799F49091690280916A029817C3
:1015A00069F490916B0280916C02981739F49091D4
:1015B0006D0280916E02981709F45BC00E949F0D26
:1015C0000E94A30D0E94080180E090E060E070E0BE
:1015D0000E94EC0180E00E94840D8FE090E060E0CA
:1015E00070E00E94EC0180E00E94840D81E060E0E8
:1015F0000E94900D8BE192E00E94B90D80919202C1
:101600000E9430080E94B90D80E061E00E94900DB8
:10161000A0919202E0919202B0E0A958BD4FF0E093
:10162000E056FD4F8C9160810E94550888E061E092
:101630000E94900DE0919202F0E0E756FD4F80810C
:10164000882319F082E292E002C08AE292E00E94CE
:10165000B90D809192028093680280916A02809312
:10166000690280916C0280936B0280916E0280937C
:101670006D0208950F931F93DF93CF93CDB7DEB71D
:1016800060970FB6F894DEBF0FBECDBF882309F474
:101690008CC00E9402010E949F0D0E94A30D0E9417
:1016A000080180E090E060E070E00E94EC0180E0E2
:1016B0000E94840D8FE090E060E070E00E94EC01F9
:1016C00080E00E94840D81E060E00E94900D8BE13B
:1016D00092E00E94B90D80916F020E9430080E9432
:1016E000B90D80E061E00E94900D8091700290E061
:1016F0008E010F5F1F4FB8014AE050E00E94620F59
:10170000C8010E94B90D85E192E00E94B90D809157
:10171000710290E0B8014AE050E00E94620FC801F7
:101720000E94B90D87E192E00E94B90D809172028A
:1017300090E0B8014AE050E00E94620FC8010E94A8
:10174000B90D82E392E00E94B90D80918F0290E082
:10175000B8014AE050E00E94620FC8010E94B90D32
:1017600080918E0290E0B8014AE050E00E94620F42
:10177000C8010E94B90D8DEA91E00E94B90D8091D7
:101780008D0290E0B8014AE050E00E94620FC8016B
:101790000E94B90D80918C0290E0B8014AE050E0BF
:1017A0000E94620FC8010E94B90D81E00E94CC0521
:1017B0008FEF91EEA4E081509040A040E1F700C08F
:1017C000000080E00E94CC058FEF91EEA4E08150F4
:1017D0009040A040E1F700C0000060960FB6F8947A
:1017E000DEBF0FBECDBFCF91DF911F910F91089546
:1017F000209197029091980281E0291709F480E0E6
:10180000909197029093980290919702992319F4DE
:101810000E949B08089590919702913019F40E94BC
:10182000A308089590919702923019F40E94EE084F
:10183000089590919702933019F40E943709089502
:1018400090919702943019F40E9480090895909124
:101850009702953019F40E944F0A089590919702CB
:101860009D3B11F40E943A0B0895809170028F5FA6
:101870008093700280917102823059F090917002D1
:10188000E0917102F0E0E358FD4F8081891770F01C
:1018900026C080917202837029F0809170028D3190
:1018A00028F41DC0809170028E31C8F091E09093B1
:1018B0007002809171028F5F80937102809171023A
:1018C0008D3068F090937102809172028F5F8093E7
:1018D000720280917202843610F0109272020E949D
:1018E0008D000E94BD0008951F920F920FB60F92B7
:1018F00011242F933F934F935F936F937F938F9315
:101900009F93AF93BF93EF93FF9380918A028F5F72
:1019100080938A0280918A028A3038F010928A027B
:1019200080918B028F5F80938B0280918B02863037
:1019300050F010928B0280918C028F5F80938C020A
:1019400081E08093960280918C028A3038F0109268
:101950008C0280918D028F5F80938D0280918D0229
:10196000863038F010928D0280918E028F5F8093C6
:101970008E0280918E028A3038F010928E02809111
:101980008F028F5F80938F0280918F02823058F098
:1019900080918E02843038F010928E0210928F0265
:1019A00081E08093950280919602882361F00E94E5
:1019B000DB0080919602882331F080919702882382
:1019C00011F01092960280919602882349F080913E
:1019D0009702882329F41092960281E00E9427043E
:1019E00080919502882321F0109295020E94350C77
:1019F000FF91EF91BF91AF919F918F917F916F91E7
:101A00005F914F913F912F910F900FBE0F901F90BC
:101A100018950E948B0584E392E00E94B90D8FEF28
:101A200093E2A4EF81509040A040E1F700C0000095
:101A30000E949F0D0E94A30D8DE492E00E94B90DBB
:101A40008FEF9BE7A2E981509040A040E1F700C0F2
:101A500000000E949F0D0E94A30D0E94240181E0BE
:101A60000E9427040E94E4070E94F80B8FEF91EE7A
:101A7000A4E081509040A040E1F700C00000F2CF08
:101A8000009711F400C008950197F1F70895449A62
:101A900000C0449808951F93662311F0459A01C031
:101AA00045983B9A3A9A399A389A40984198429880
:101AB000439887FD409A182F86FD419A15FD429A5A
:101AC00014FD439A0E94470D4098419842984398CC
:101AD00013FD409A12FD419A11FD429A10FD439A5E
:101AE0000E94470D439A429A419A409A1F91089545
:101AF0001F93182F80EA9FE00E94400D812F60E025
:101B00000E944B0D1F9108951F93182F80EA9FE0AC
:101B10000E94400D812F61E00E944B0D1F9108959E
:101B2000662311F4805801C080540E94780D0895F6
:101B300080EA9FE00E94400D81E090E0089581E0FE
:101B40000E94780D089582E00E94780D08951F93F9
:101B5000182F80EA9FE00E94400D1A3021F480EC9B
:101B60000E94780D04C0812F61E00E944B0D1F91EF
:101B70000895CF93DF93EC0102C00E94A70D8991D5
:101B80008823D9F7DF91CF910895CF93DF93EC01AC
:101B900002C00E94A70DFE01219684918823C9F7F7
:101BA000DF91CF9108951F93182F3D9A3C9A3B9A4D
:101BB0003A9A399A389A80E09AEF0E94400D429AF8
:101BC000439A0E94470D80E09EE40E94400D0E94CF
:101BD000470D80E091E00E94400D0E94470D80E09B
:101BE00091E00E94400D43980E94470D80E091E0F3
:101BF0000E94400D88E20E94780D88E00E94780DD6
:101C00000E949F0D86E00E94780D812F0E94780D22
:101C10001F9108958EB180728EB98EB180718EB988
:101C20006D986C9808956C9880E590E0FC01319770
:101C3000F1F76D9A0197F1F708956D9A80E590E0BC
:101C4000FC013197F1F76C98E0E3F0E03197F1F7A0
:101C50006D980197F1F7089598E040E350E020E592
:101C600030E06C9AFA013197F1F787FF02C06D9866
:101C700001C06D9AF9013197F1F76C98F90131972C
:101C8000F1F7649BFECF915011F0880FEACF6C9A68
:101C900080E390E00197F1F76D9880E590E0FC011A
:101CA0003197F1F76C98FC013197F1F72CB16C9AF0
:101CB0000197F1F781E025FD80E00895982F20E05D
:101CC00030E080E040E550E060E870E06C9AFA01B6
:101CD0003197F1F76C98FA013197F1F7649BFECFD9
:101CE000659B08C0FB01022E02C0F595E7950A949A
:101CF000E2F78E2B2F5F3F4F2830310539F76C9A72
:101D0000E0E3F0E03197F1F7992311F06D9A01C00B
:101D10006D9820E530E0F9013197F1F76C98F90101
:101D20003197F1F76C9AF9013197F1F76D980895B1
:101D30001F93DF93CF9300D000D00F92CDB7DEB7C3
:101D4000182FFE01319685E0DF011D928A95E9F793
:101D5000989AA09A8FEF91EEA4E081509040A04015
:101D6000E1F700C00000A0988FEF90EEA0E0815056
:101D70009040A040E1F700C00000A09A95E09A953D
:101D8000F1F700009898A0EDAA95F1F7909953C04B
:101D90008FE391E00197F1F700C00000909B4BC0EA
:101DA000AFE3B1E01197F1F700C00000BE016A5F38
:101DB0007F4F41E050E01BC0909BFECFB0EABA9548
:101DC000F1F7909B08C0DA01022E02C0AA0FBB1FD8
:101DD0000A94E2F79A2B9099FECF215030408FEF72
:101DE0002F3F380749F79193E617F70721F027E0CF
:101DF00030E090E0E1CF989AA09A8FEF91EEA4E0C6
:101E000081509040A040E1F700C0000089819B8193
:101E10004A81282F30E0240F311D290F311D4C81BC
:101E2000240F311D4D8150E02417350721F4112373
:101E300021F0113019F08FEF01C0892F0F900F9012
:101E40000F900F900F90CF91DF911F91089580E038
:101E50000E94980E089581E00E94980E0895991BA3
:101E600079E004C0991F961708F0961B881F7A9591
:101E7000C9F78095089597FB092E07260AD077FDAC
:101E800004D00CD006D000201AF4709561957F4FD5
:101E90000895F6F7909581959F4F0895AA1BBB1B57
:101EA00051E107C0AA1FBB1FA617B70710F0A61B5A
:101EB000B70B881F991F5A95A9F780959095BC017B
:101EC000CD010895FB019F01E8944230C4F04532F2
:101ED000B4F44A3029F497FB1EF4909581959F4FF6
:101EE000642F77270E944E0F805D8A330CF0895D46
:101EF0008193CB010097A1F716F45DE25193108214
:101F0000C9010C94980FF999FECF92BD81BDF89A42
:101F1000992780B50895262FF999FECF92BD81BDEE
:101F200020BD0FB6F894FA9AF99A0FBE019608955B
:101F3000DC01FC01672F71917723E1F7329704C030
:101F40007C916D9370836291AE17BF07C8F30895BB
:041F5000F894FFCF33
:101F540020202020204E6564656C612020202020F4
:101F64000020202020506F6E64656C6F6B20202051
:101F74002000202020202055746F726F6B202020B9
:101F840020200020202020205374726564612020CA
:101F940020202000202020202053747672746F6B40
:101FA40020202020002020202020506961746F6BA5
:101FB4002020202020002020202020536F626F74D6
:101FC400612020202020004E6564656C6100506F04
:101FD4006E64656C6F6B0055746F726F6B00537435
:101FE400726564610053747672746F6B005069613A
:101FF400746F6B00536F626F74610030003A005469
:1020040065706C6F74613A20202020430A566C6816
:102014006B6F73743A2020202025004D617854653D
:10202400706C6F74613A20202020430A4D61785609
:102034006C686B6F73743A2020202025004D696E04
:102044005465706C6F74613A20202020430A4D69F6
:102054006E566C686B6F73743A2020202025000A3A
:1020640020202020002E002E323000427564696B3F
:102074002D005A41504E555459005659504E5554FE
:1020840059002D004E697472616D3134370A5465FC
:10209400706C6F566C686B6F2D6D6572005665724F
:1020A4007A696120627564696B0A56656C6B652098
:1020B400686F64696E79000C09FFFFFFFFFFFF067C
:1020C40019070F090909090C0C0C0C0C0C0C1F1C2A
:0A20D4001F1E1F1E1F1F1E1F1E1FD0
:00000001FF
